:100000000C9462000C948A000C948A000C948A0070
:100010000C948A000C948A000C948A000C948A0038
:100020000C948A000C948A000C948A000C948A0028
:100030000C948A000C948A000C948A000C948A0018
:100040000C9477020C948A000C949E030C948A0002
:100050000C948A000C948A000C948A000C948A00F8
:100060000C948A000C948A000000000024002700F1
:100070002A0000000000250028002B0000000000DE
:1000800023002600290004040404040404040202DA
:100090000202020203030303030301020408102007
:1000A0004080010204081020010204081020000012
:1000B0000007000201000003040600000000000029
:1000C0000000230511241FBECFEFD4E0DEBFCDBF5B
:1000D00011E0A0E0B1E0E6EEFDE002C005900D9277
:1000E000AA31B107D9F713E0AAE1B1E001C01D922E
:1000F000AC30B107E1F710E0C4ECD0E004C02297C7
:10010000FE010E94ED06C23CD107C9F70E947002B1
:100110000C94F1060C94000089EF92E040E051EE5F
:1001200060E070E00E94DB0364E670E080E090E055
:100130000E94BF028091000161E00E943103809122
:10014000020161E00E9431038091040161E00E949C
:1001500031038091020160E00E945103809104010B
:1001600061E00E9451030895BF92CF92DF92EF9217
:10017000FF920F931F93DF93CF93CDB7DEB72A97EC
:100180000FB6F894DEBF0FBECDBF6B01DE01119636
:10019000E6E0F1E02AE001900D922150E1F79C01A8
:1001A0008A579F4FFC01849126563F4FF901B49026
:1001B000E82FF0E0EE0FFF1FEC0FFD1F0181128111
:1001C00090E2E92EF12CE00EF11EF80180A18B29BE
:1001D00080A38AE090E00E94E902F894F80180A1EF
:1001E0009B2D9095892380A3000000000000000053
:1001F00000000000000000000000000000000000FF
:1002000000000000000000000000000000000000EE
:1002100000000000000000000000000000000000DE
:1002200000000000000000000000000000000000CE
:1002300000000000000000000000000000000000BE
:10024000000000000000000020E030E0C0FE04C01C
:10025000F70180818B2903C0F70180818923808386
:10026000000000000000000000000000000000008E
:10027000000000000000000000000000000000007E
:10028000000000000000000000000000000000006E
:10029000000000000000000000000000000000005E
:1002A000000000000000000000000000000000004E
:1002B000000000000000000000000000000000003E
:1002C0002F5F3F4F2830310519F0D594C794BECF2A
:1002D000F80180A18B2980A378942A960FB6F89410
:1002E000DEBF0FBECDBFCF91DF911F910F91FF9069
:1002F000EF90DF90CF90BF900895CF93DF938091E0
:10030000000160E00E94510384E690E00E94E9024F
:1003100010922C02C0E0D0E0809100019091010188
:10032000C034D10531F0FE01E45DFD4F608170E025
:1003300002C060E070E00E94B4002196C134D10593
:1003400059F7DF91CF9108958091040161E00E94F7
:10035000510389EF92E00E94D404882309F49CC0E1
:1003600089EF92E00E94E804AC0190931B01809316
:100370001A01893D910549F480911C0190911D015C
:10038000892B19F481E090E00BC020911C01309181
:100390001D012130310549F44093210182E090E0B4
:1003A00090931D0180931C010EC0C9010297049710
:1003B00050F4F901EE5DFE4F40832F5F3F4F3093C5
:1003C0001D0120931C0180911C0190911D01069735
:1003D00009F062C08091040160E00E945103109214
:1003E0001D0110921C015091240130912501209192
:1003F0002601832F850F820F809320019091270182
:1004000040912101981741F4E42FF0E0E45DFE4FA4
:1004100050833183228340C050E060E070E089EF78
:1004200092E020E030E00E9453064091240150E029
:1004300060E070E089EF92E020E030E00E94530637
:100440004091250150E060E070E089EF92E020E00B
:1004500030E00E9453064091260150E060E070E0D9
:1004600089EF92E020E030E00E945306409127019E
:1004700050E060E070E089EF92E020E030E00E9420
:1004800053064091200150E060E070E089EF92E077
:1004900020E030E00E94530680911C0190911D01E4
:1004A000892BE9F48091210190E0DC01A45DBE4F2D
:1004B000AC014E5F5F4F0AC0E82F2C91803420F4CE
:1004C000F0E0E45DFD4F208301961196481759072F
:1004D0009CF790931F0180931E010E947D01089557
:1004E0000E94F7020E948C000E94A401FDCF1F927F
:1004F0000F920FB60F9211242F933F938F939F93D8
:10050000AF93BF938091700290917102A09172029B
:10051000B0917302309174020196A11DB11D232F79
:100520002D5F2D3720F02D570196A11DB11D209371
:1005300074028093700290937102A0937202B09340
:10054000730280916C0290916D02A0916E02B09145
:100550006F020196A11DB11D80936C0290936D02F4
:10056000A0936E02B0936F02BF91AF919F918F9154
:100570003F912F910F900FBE0F901F901895EF9203
:10058000FF920F931F937B018C018FB7F8944091DA
:1005900070025091710260917202709173028FBF6C
:1005A0002FB7F8948091700290917102A09172021D
:1005B000B09173022FBF841B950BA60BB70BE816E7
:1005C000F9060A071B0760F71F910F91FF90EF9044
:1005D0000895019759F0FC01EE0FFF1FEE0FFF1F6A
:1005E00032978FB7F8943197F1F78FBF08957894C9
:1005F00084B5826084BD84B5816084BD85B5826028
:1006000085BD85B5816085BDEEE6F0E080818160C5
:100610008083E1E8F0E08081826080838081816076
:100620008083E0E8F0E0808181608083E1EBF0E0AE
:10063000808184608083E0EBF0E080818160808352
:10064000EAE7F0E08081846080838081826080833B
:100650008081816080838081806880831092C10066
:100660000895282F30E0C90186569F4FFC019491D0
:100670002A573F4FF9018491882391F0E82FF0E049
:10068000EE0FFF1FE859FF4FA591B491662329F49F
:100690008C91909589238C9308958C91892B8C93C0
:1006A0000895482F50E0CA0182559F4FFC012491C4
:1006B000CA0186569F4FFC0194914A575F4FFA0139
:1006C00034913323D1F1222331F1233021F480916D
:1006D00080008F7705C0243031F4809180008F7DB9
:1006E0008093800018C0213019F484B58F7704C03E
:1006F000223021F484B58F7D84BD0DC0263021F4D5
:100700008091B0008F7705C0273029F48091B00028
:100710008F7D8093B000E32FF0E0EE0FFF1FEE58C7
:10072000FF4FA591B491662329F48C91909589236C
:100730008C9308958C91892B8C9308951F920F921E
:100740000FB60F9211242F933F934F935F936F93A4
:100750007F938F939F93AF93BF93EF93FF934091BA
:10076000C600E091F502F091F602CF01019660E833
:1007700070E00E9487069C018091F7029091F80238
:100780002817390739F0EB58FD4F40833093F602B4
:100790002093F502FF91EF91BF91AF919F918F91BF
:1007A0007F916F915F914F913F912F910F900FBE6D
:1007B0000F901F9018955F926F927F928F929F92E9
:1007C000AF92BF92CF92DF92EF92FF920F931F935F
:1007D000CF93DF93EC013A014B01413482E4580797
:1007E0008FE0680780E078070CF07FC060E874E86D
:1007F0008EE190E0A40193010E94BC06215030409C
:1008000040405040CA01B90122E030E040E050E0F1
:100810000E94BC0659016A01A601950120953095F8
:100820004095509594E0220F331F441F551F9A9511
:10083000D1F760E074E284EF90E00E94BC06CA0148
:10084000B9012FEF30E040E050E00E946806A401BB
:1008500093010E94BC06C90181509F4F18161906CA
:100860001CF4522E5A9403C055245394521A60E03B
:1008700079E08DE390E0A40193010E94BC06215031
:10088000304040405040CA01B90122E030E040E031
:1008900050E00E94BC06209530954095509583E02D
:1008A000220F331F441F551F8A95D1F760E074E271
:1008B00084EF90E00E94BC06CA01B9012FEF30E03E
:1008C00040E050E00E946806A40193010E94BC062B
:1008D000C90181509F4F181619061CF4822F8150B0
:1008E00002C081E0821B851500F5E885F98581E06D
:1008F00090E00A8802C0880F991F0A94E2F780836B
:1009000060E079E08DE390E0A40193010E94BC06D1
:100910002150304040405040CA01B90122E030E04F
:1009200040E050E00E94BC0604C0E885F9851082D2
:100930009501EC81FD813083EE81FF812083EA8582
:10094000FB85208141E050E0CA010E8402C0880F7F
:10095000991F0A94E2F7282B2083EA85FB852081E2
:10096000CA010F8402C0880F991F0A94E2F7282B4E
:100970002083EA85FB858081088802C0440F551FCB
:100980000A94E2F7842B8083DF91CF911F910F911E
:10099000FF90EF90DF90CF90BF90AF909F908F909F
:1009A0007F906F905F900895DC011296ED91FC911D
:1009B0001397E058FF4F8191919180589F4F20816C
:1009C0003181821B930B60E870E00E9487060895D6
:1009D000CF93DF93DC011296ED91FC911397EF0119
:1009E000CE57DF4F48815981E058FF4F8081918178
:1009F000E058F0408417950719F42FEF3FEF0CC033
:100A0000E40FF51F2081CA01019660E870E00E94A2
:100A100087069983888330E0C901DF91CF910895DB
:100A2000FC01A085B18521898C9190E0022E02C045
:100A3000959587950A94E2F780FFF6CF0484F585B3
:100A4000E02D6083089584E191E09093FA02809311
:100A5000F90285E792E09093FC028093FB0285EC1B
:100A600090E09093FE028093FD0284EC90E09093DE
:100A700000038093FF0280EC90E090930203809348
:100A8000010381EC90E0909304038093030386ECD0
:100A900090E0909306038093050384E0809307031E
:100AA00083E08093080387E08093090385E08093C7
:100AB0000A0381E080930B0308950F931F93CF9354
:100AC000DF938C01EB0109C02196D801ED91FC91D7
:100AD0000190F081E02DC801099568816623A1F796
:100AE000DF91CF911F910F910895EF92FF920F9395
:100AF0001F93CF93DF938C017B01EA010CC0D701D8
:100B00006D917D01D801ED91FC910190F081E02D76
:100B1000C80109952197209791F7DF91CF911F91F7
:100B20000F91FF90EF9008952F923F924F925F9216
:100B30006F927F928F929F92AF92BF92CF92DF92ED
:100B4000EF92FF920F931F93DF93CF93CDB7DEB752
:100B5000A0970FB6F894DEBF0FBECDBF1C016A018F
:100B60007B01411551056105710549F4DC01ED91E9
:100B7000FC910190F081E02D60E3099554C0882438
:100B800099245401422E55246624772401E010E074
:100B90000C0F1D1F080D191DC701B601A3019201FD
:100BA0000E949A06F80160830894811C911CA11C84
:100BB000B11CC701B601A30192010E949A06C901A6
:100BC000DA016C017D01C114D104E104F104F1F6F4
:100BD00081E0E82EF12CEC0EFD1EE80CF91C3E0124
:100BE0000894611C711CD501C4010197A109B109C8
:100BF0006C01C818D90814C0F601EE0DFF1D608104
:100C00006A3010F4605D01C0695CD101ED91FC9126
:100C10000190F081E02DC10109950894E108F108E7
:100C20006E147F0449F7A0960FB6F894DEBF0FBE8E
:100C3000CDBFCF91DF911F910F91FF90EF90DF908B
:100C4000CF90BF90AF909F908F907F906F905F906C
:100C50004F903F902F900895EF92FF920F931F9324
:100C6000CF93DF93EC017A018B0177FF0FC0E8810E
:100C7000F9810190F081E02D6DE2099510950095C4
:100C8000F094E094E11CF11C011D111DCE01B8018E
:100C9000A7012AE00E949405DF91CF911F910F9147
:100CA000FF90EF900895DC012115310541F4ED919D
:100CB000FC910190F081E02D642F099508952A3070
:100CC000310519F40E942C0608950E949405089598
:100CD000629FD001739FF001829FE00DF11D649F20
:100CE000E00DF11D929FF00D839FF00D749FF00DAC
:100CF000659FF00D9927729FB00DE11DF91F639F4D
:100D0000B00DE11DF91FBD01CF011124089597FB1E
:100D1000092E07260AD077FD04D049D006D000203E
:100D20001AF4709561957F4F0895F6F79095819527
:100D30009F4F0895A1E21A2EAA1BBB1BFD010DC0F7
:100D4000AA1FBB1FEE1FFF1FA217B307E407F5077B
:100D500020F0A21BB30BE40BF50B661F771F881F57
:100D6000991F1A9469F760957095809590959B01ED
:100D7000AC01BD01CF01089597FB092E05260ED0C9
:100D800057FD04D0D7DF0AD0001C38F450954095A9
:100D9000309521953F4F4F4F5F4F0895F6F790954F
:100DA0008095709561957F4F8F4F9F4F0895AA1B37
:100DB000BB1B51E107C0AA1FBB1FA617B70710F046
:100DC000A61BB70B881F991F5A95A9F78095909578
:100DD000BC01CD010895EE0FFF1F0590F491E02DA9
:060DE0000994F894FFCF16
:100DE60005000C000D0000000000050008000B00C7
:0A0DF6000000000010055D05750502
:00000001FF
